
 RPC16C8

 Start     Length     Name                   Class
 0001:0000 00000H     CLNTVNS_TEXT           CODE
 0001:0000 00000H     LTSTART_TEXT           CODE
 0001:0000 001CBH     _TEXT                  CODE
 0001:01D0 00CC4H     COMDAT_SEG1            CODE
 0002:0000 00038H     _DATA                  DATA
 0002:0038 00000H     CONST                  CONST
 0002:0038 00000H     _BSS                   BSS
 0002:0040 00012H     c_common               BSS

 Origin   Group
 0002:0   DGROUP

 Address   Export                  Alias

 0001:07B2 CLIENTCLOSE             CLIENTCLOSE
 0001:062A CLIENTOPEN              CLIENTOPEN
 0001:097A CLIENTRECV              CLIENTRECV
 0001:08D2 CLIENTSEND              CLIENTSEND
 0001:0B28 CLIENTTOWERCONSTRUCT    CLIENTTOWERCONSTRUCT
 0001:0C66 CLIENTTOWEREXPLODE      CLIENTTOWEREXPLODE
 0001:0274 INSERTCONN              INSERTCONN
 0001:01D0 INSERTTASK              INSERTTASK
 0001:02C4 REMOVECONN              REMOVECONN
 0001:0220 REMOVETASK              REMOVETASK
 0001:0D60 TRANSPORTLOAD           TRANSPORTLOAD
 0001:0014 WEP                     WEP

  Address         Publics by Name

 0001:0E72       ??_C@_03GEHA@385?$AA@
 0001:0E62       ??_C@_07LDNL@RPC?5VNS?$AA@
 0001:0E6A       ??_C@_07MKKD@CLNTVNS?$AA@
 0001:0E84       ??_C@_0BA@CFLE@VM_SOCKETNOTIFY?$AA@
 0001:0E76       ??_C@_0O@IPEE@ncacn_vns_spp?$AA@
 0001:0894       ASYNCEVENTPROC
 0001:07B2       CLIENTCLOSE
 0001:062A       CLIENTOPEN
 0001:097A       CLIENTRECV
 0001:08D2       CLIENTSEND
 0001:0B28       CLIENTTOWERCONSTRUCT
 0001:0C66       CLIENTTOWEREXPLODE
 0001:03CA       CLNTVNSCLEANUP
 0000:0000  Imp  CREATEWINDOW         (USER.41)
 0000:0000  Imp  DEFWINDOWPROC        (USER.107)
 0000:0000  Imp  DISPATCHMESSAGE      (USER.114)
 0000:0000  Imp  GETCURRENTTASK       (KERNEL.36)
 0000:0000  Imp  GETCURRENTTIME       (USER.15)
 0000:0000  Imp  GETSTOCKOBJECT       (GDI.87)
 0001:0274       INSERTCONN
 0001:01D0       INSERTTASK
 0001:0000       LIBENTRY
 0000:0000  Imp  LOADCURSOR           (USER.173)
 0000:0000  Imp  LOCALINIT            (KERNEL.4)
 0001:0E5C       MYWEP
 0000:0000  Imp  PEEKMESSAGE          (USER.109)
 0000:0000  Imp  REGISTERCLASS        (USER.57)
 0000:0000  Imp  REGISTERWINDOWMESSAGE (USER.118)
 0001:02C4       REMOVECONN
 0001:0220       REMOVETASK
 0000:0000  Imp  SHOWWINDOW           (USER.42)
 0000:0000  Imp  TRANSLATEMESSAGE     (USER.113)
 0001:0D60       TRANSPORTLOAD
 0000:0000  Imp  UPDATEWINDOW         (USER.124)
 0000:0000  Imp  VNSCLOSESOCKET       (VNSAPI.14)
 0000:0000  Imp  VNSDONE              (VNSAPI.163)
 0000:0000  Imp  VNSENDSTSESSION      (VNSAPI.513)
 0000:0000  Imp  VNSGETSSPPPORT       (VNSAPI.417)
 0000:0000  Imp  VNSOPENSOCKET        (VNSAPI.10)
 0000:0000  Imp  VNSSOCKETNOTIFYWINDOW (VNSAPI.20)
 0000:0000  Imp  VNSSOCKETRECEIVE     (VNSAPI.11)
 0000:0000  Imp  VNSSOCKETSEND        (VNSAPI.12)
 0000:0000  Imp  VNSSOCKETWAIT        (VNSAPI.13)
 0000:0000  Imp  VNSSTARTSTSESSION    (VNSAPI.542)
 0001:0014       WEP
 0002:0046       _AsyncCallComplete
 0001:004C       _atoi
 0001:04D8       _BlockForRecv
 0001:0834       _CheckForCompletion
 0002:0034       _DllTermination
 0002:0042       _HeadConn
 0002:004E       _HeadTask
 0002:0032       _hInstanceDLL
 0001:0582       _LocalBlockForSendRecv
 0001:0406       _MayBeCreateWindow
 0002:004A       _RpcRuntimeInfo
 0001:0032       _strlen
 0002:0002       _TransInfo
 0002:0040       _VM_SocketNotify
 0001:031E       _VnsFindConn
 0001:0376       _VnsFindWindowByTask
 0002:0000       _VNS_Verbose
 0000:0000  Imp  __AHINCR             (KERNEL.114)
 0001:0112       __catox
 0001:0168       __cltoasub
 0001:0175       __cxtoa
 0001:006C       __fmemcpy
 0001:00CA       __fmemset
 0001:0050       __itoa

  Address         Publics by Value

 0000:0000  Imp  PEEKMESSAGE          (USER.109)
 0000:0000  Imp  VNSSOCKETNOTIFYWINDOW (VNSAPI.20)
 0000:0000  Imp  REGISTERCLASS        (USER.57)
 0000:0000  Imp  VNSENDSTSESSION      (VNSAPI.513)
 0000:0000  Imp  REGISTERWINDOWMESSAGE (USER.118)
 0000:0000  Imp  SHOWWINDOW           (USER.42)
 0000:0000  Imp  UPDATEWINDOW         (USER.124)
 0000:0000  Imp  DISPATCHMESSAGE      (USER.114)
 0000:0000  Imp  VNSSOCKETSEND        (VNSAPI.12)
 0000:0000  Imp  GETSTOCKOBJECT       (GDI.87)
 0000:0000  Imp  VNSGETSSPPPORT       (VNSAPI.417)
 0000:0000  Imp  LOADCURSOR           (USER.173)
 0000:0000  Imp  DEFWINDOWPROC        (USER.107)
 0000:0000  Imp  VNSSOCKETRECEIVE     (VNSAPI.11)
 0000:0000  Imp  VNSDONE              (VNSAPI.163)
 0000:0000  Imp  VNSSOCKETWAIT        (VNSAPI.13)
 0000:0000  Imp  LOCALINIT            (KERNEL.4)
 0000:0000  Imp  VNSSTARTSTSESSION    (VNSAPI.542)
 0000:0000  Imp  VNSOPENSOCKET        (VNSAPI.10)
 0000:0000  Imp  __AHINCR             (KERNEL.114)
 0000:0000  Imp  VNSCLOSESOCKET       (VNSAPI.14)
 0000:0000  Imp  CREATEWINDOW         (USER.41)
 0000:0000  Imp  GETCURRENTTIME       (USER.15)
 0000:0000  Imp  GETCURRENTTASK       (KERNEL.36)
 0000:0000  Imp  TRANSLATEMESSAGE     (USER.113)
 0001:0000       LIBENTRY
 0001:0014       WEP
 0001:0032       _strlen
 0001:004C       _atoi
 0001:0050       __itoa
 0001:006C       __fmemcpy
 0001:00CA       __fmemset
 0001:0112       __catox
 0001:0168       __cltoasub
 0001:0175       __cxtoa
 0001:01D0       INSERTTASK
 0001:0220       REMOVETASK
 0001:0274       INSERTCONN
 0001:02C4       REMOVECONN
 0001:031E       _VnsFindConn
 0001:0376       _VnsFindWindowByTask
 0001:03CA       CLNTVNSCLEANUP
 0001:0406       _MayBeCreateWindow
 0001:04D8       _BlockForRecv
 0001:0582       _LocalBlockForSendRecv
 0001:062A       CLIENTOPEN
 0001:07B2       CLIENTCLOSE
 0001:0834       _CheckForCompletion
 0001:0894       ASYNCEVENTPROC
 0001:08D2       CLIENTSEND
 0001:097A       CLIENTRECV
 0001:0B28       CLIENTTOWERCONSTRUCT
 0001:0C66       CLIENTTOWEREXPLODE
 0001:0D60       TRANSPORTLOAD
 0001:0E5C       MYWEP
 0001:0E62       ??_C@_07LDNL@RPC?5VNS?$AA@
 0001:0E6A       ??_C@_07MKKD@CLNTVNS?$AA@
 0001:0E72       ??_C@_03GEHA@385?$AA@
 0001:0E76       ??_C@_0O@IPEE@ncacn_vns_spp?$AA@
 0001:0E84       ??_C@_0BA@CFLE@VM_SOCKETNOTIFY?$AA@
 0002:0000       _VNS_Verbose
 0002:0002       _TransInfo
 0002:0032       _hInstanceDLL
 0002:0034       _DllTermination
 0002:0040       _VM_SocketNotify
 0002:0042       _HeadConn
 0002:0046       _AsyncCallComplete
 0002:004A       _RpcRuntimeInfo
 0002:004E       _HeadTask

Program entry point at 0001:0000
